

Microchip MPLAB XC8 Assembler V2.32 build 20210201212658 
                                                                                               Mon Jan 17 12:07:46 2022

Microchip MPLAB XC8 C Compiler v2.32 (Free license) build 20210201212658 Og1 
     1                           	processor	18F4580
     2                           	fnconf	rparam,??,?,0
     3                           	pagewidth 120
     4                           	opt	flic
     5                           	psect	cinit,global,reloc=2,class=CODE,delta=1
     6                           	psect	cstackCOMRAM,global,class=COMRAM,space=1,delta=1,lowdata,noexec
     7                           	psect	text0,global,reloc=2,class=CODE,delta=1
     8                           	psect	text1,global,reloc=2,class=CODE,delta=1
     9                           	psect	intcode,global,reloc=2,class=CODE,delta=1
    10                           	psect	intcode_body,global,reloc=2,class=CODE,delta=1
    11                           	psect	intsave_regs,global,class=BIGRAM,space=1,delta=1,noexec
    12                           	psect	rparam,global,class=COMRAM,space=1,delta=1,noexec
    13                           	psect	temp,global,ovrld,common,class=COMRAM,space=1,delta=1
    14                           	psect	idloc,global,abs,ovrld,class=IDLOC,space=5,delta=1,noexec
    15                           	psect	config,global,abs,ovrld,class=CONFIG,space=4,delta=1,noexec
    16  0000                     
    17                           ; Version 2.40
    18                           ; Generated 17/11/2021 GMT
    19                           ; 
    20                           ; Copyright © 2021, Microchip Technology Inc. and its subsidiaries ("Microchip")
    21                           ; All rights reserved.
    22                           ; 
    23                           ; This software is developed by Microchip Technology Inc. and its subsidiaries ("Microch
      +                          ip").
    24                           ; 
    25                           ; Redistribution and use in source and binary forms, with or without modification, are
    26                           ; permitted provided that the following conditions are met:
    27                           ; 
    28                           ;     1. Redistributions of source code must retain the above copyright notice, this lis
      +                          t of
    29                           ;        conditions and the following disclaimer.
    30                           ; 
    31                           ;     2. Redistributions in binary form must reproduce the above copyright notice, this 
      +                          list
    32                           ;        of conditions and the following disclaimer in the documentation and/or other
    33                           ;        materials provided with the distribution. Publication is not required when
    34                           ;        this file is used in an embedded application.
    35                           ; 
    36                           ;     3. Microchip's name may not be used to endorse or promote products derived from th
      +                          is
    37                           ;        software without specific prior written permission.
    38                           ; 
    39                           ; THIS SOFTWARE IS PROVIDED BY MICROCHIP "AS IS" AND ANY EXPRESS OR IMPLIED WARRANTIES,
    40                           ; INCLUDING, BUT NOT LIMITED TO, THE IMPLIED WARRANTIES OF MERCHANTABILITY AND FITNESS F
      +                          OR
    41                           ; PURPOSE ARE DISCLAIMED.  IN NO EVENT SHALL MICROCHIP BE LIABLE FOR ANY DIRECT, INDIREC
      +                          T,
    42                           ; INCIDENTAL, SPECIAL, EXEMPLARY, OR CONSEQUENTIAL DAMAGES (INCLUDING BUT NOT LIMITED TO
    43                           ; PROCUREMENT OF SUBSTITUTE GOODS OR SERVICES; LOSS OF USE, DATA OR PROFITS; OR BUSINESS
    44                           ; INTERRUPTION) HOWSOEVER CAUSED AND ON ANY THEORY OF LIABILITY, WHETHER IN CONTRACT, ST
      +                          RICT
    45                           ; LIABILITY, OR TORT (INCLUDING NEGLIGENCE OR OTHERWISE) ARISING IN ANY WAY OUT OF THE U
      +                          SE OF
    46                           ; THIS SOFTWARE, EVEN IF ADVISED OF THE POSSIBILITY OF SUCH DAMAGE.
    47                           ; 
    48                           ; 
    49                           ; Code-generator required, PIC18F4580 Definitions
    50                           ; 
    51                           ; SFR Addresses
    52  0000                     _PORTA	set	3968
    53  0000                     _PORTC	set	3970
    54  0000                     _ADCON1	set	4033
    55  0000                     _TRISC	set	3988
    56  0000                     _TRISA	set	3986
    57  0000                     _INT0IF	set	32657
    58  0000                     _PEIE	set	32662
    59  0000                     _INT0IE	set	32660
    60  0000                     _GIEH	set	32663
    61                           
    62                           ; #config settings
    63                           
    64                           	psect	cinit
    65  000092                     __pcinit:
    66                           	callstack 0
    67  000092                     start_initialization:
    68                           	callstack 0
    69  000092                     __initialization:
    70                           	callstack 0
    71  000092                     end_of_initialization:
    72                           	callstack 0
    73  000092                     __end_of__initialization:
    74                           	callstack 0
    75  000092  9006               	bcf	int$flags,0,c	;clear compiler interrupt flag (level 1)
    76  000094  9206               	bcf	int$flags,1,c	;clear compiler interrupt flag (level 2)
    77  000096  0100               	movlb	0
    78  000098  EF09  F000         	goto	_main	;jump to C main() function
    79                           
    80                           	psect	cstackCOMRAM
    81  000001                     __pcstackCOMRAM:
    82                           	callstack 0
    83  000001                     delay@ms:
    84                           	callstack 0
    85                           
    86                           ; 2 bytes @ 0x0
    87  000001                     	ds	2
    88  000003                     ??_delay:
    89                           
    90                           ; 1 bytes @ 0x2
    91  000003                     	ds	1
    92  000004                     delay@i:
    93                           	callstack 0
    94                           
    95                           ; 2 bytes @ 0x3
    96  000004                     	ds	2
    97  000006                     
    98                           ; 1 bytes @ 0x5
    99 ;;
   100 ;;Main: autosize = 0, tempsize = 0, incstack = 0, save=0
   101 ;;
   102 ;; *************** function _main *****************
   103 ;; Defined at:
   104 ;;		line 3 in file "interrupt.c"
   105 ;; Parameters:    Size  Location     Type
   106 ;;		None
   107 ;; Auto vars:     Size  Location     Type
   108 ;;		None
   109 ;; Return value:  Size  Location     Type
   110 ;;                  1    wreg      void 
   111 ;; Registers used:
   112 ;;		wreg, status,2, status,0, cstack
   113 ;; Tracked objects:
   114 ;;		On entry : 0/0
   115 ;;		On exit  : 0/0
   116 ;;		Unchanged: 0/0
   117 ;; Data sizes:     COMRAM   BANK0   BANK1   BANK2   BANK3   BANK4   BANK5
   118 ;;      Params:         0       0       0       0       0       0       0
   119 ;;      Locals:         0       0       0       0       0       0       0
   120 ;;      Temps:          0       0       0       0       0       0       0
   121 ;;      Totals:         0       0       0       0       0       0       0
   122 ;;Total ram usage:        0 bytes
   123 ;; Hardware stack levels required when called: 2
   124 ;; This function calls:
   125 ;;		_delay
   126 ;; This function is called by:
   127 ;;		Startup code after reset
   128 ;; This function uses a non-reentrant model
   129 ;;
   130                           
   131                           	psect	text0
   132  000012                     __ptext0:
   133                           	callstack 0
   134  000012                     _main:
   135                           	callstack 29
   136  000012                     
   137                           ;interrupt.c: 4:     TRISA=0x00;
   138  000012  0E00               	movlw	0
   139  000014  6E92               	movwf	146,c	;volatile
   140                           
   141                           ;interrupt.c: 5:     TRISC=0x00;
   142  000016  0E00               	movlw	0
   143  000018  6E94               	movwf	148,c	;volatile
   144                           
   145                           ;interrupt.c: 6:     ADCON1=0x0f;
   146  00001A  0E0F               	movlw	15
   147  00001C  6EC1               	movwf	193,c	;volatile
   148  00001E                     
   149                           ;interrupt.c: 7:     GIEH=1;
   150  00001E  8EF2               	bsf	4082,7,c	;volatile
   151  000020                     
   152                           ;interrupt.c: 8:     INT0IE=1;
   153  000020  88F2               	bsf	4082,4,c	;volatile
   154  000022                     
   155                           ;interrupt.c: 9:     PEIE=1;
   156  000022  8CF2               	bsf	4082,6,c	;volatile
   157  000024                     l25:
   158                           
   159                           ;interrupt.c: 11:         PORTC=0x00;
   160  000024  0E00               	movlw	0
   161  000026  6E82               	movwf	130,c	;volatile
   162  000028                     
   163                           ;interrupt.c: 12:         delay(100);
   164  000028  0E00               	movlw	0
   165  00002A  6E02               	movwf	(delay@ms+1)^0,c
   166  00002C  0E64               	movlw	100
   167  00002E  6E01               	movwf	delay@ms^0,c
   168  000030  EC25  F000         	call	_delay	;wreg free
   169  000034                     
   170                           ;interrupt.c: 13:         PORTC=0xff;
   171  000034  6882               	setf	130,c	;volatile
   172  000036                     
   173                           ;interrupt.c: 14:         delay(100);
   174  000036  0E00               	movlw	0
   175  000038  6E02               	movwf	(delay@ms+1)^0,c
   176  00003A  0E64               	movlw	100
   177  00003C  6E01               	movwf	delay@ms^0,c
   178  00003E  EC25  F000         	call	_delay	;wreg free
   179  000042  EF12  F000         	goto	l25
   180  000046  EF07  F000         	goto	start
   181  00004A                     __end_of_main:
   182                           	callstack 0
   183                           
   184 ;; *************** function _delay *****************
   185 ;; Defined at:
   186 ;;		line 24 in file "interrupt.c"
   187 ;; Parameters:    Size  Location     Type
   188 ;;  ms              2    0[COMRAM] int 
   189 ;; Auto vars:     Size  Location     Type
   190 ;;  i               2    3[COMRAM] int 
   191 ;; Return value:  Size  Location     Type
   192 ;;                  1    wreg      void 
   193 ;; Registers used:
   194 ;;		wreg, status,2, status,0
   195 ;; Tracked objects:
   196 ;;		On entry : 0/0
   197 ;;		On exit  : 0/0
   198 ;;		Unchanged: 0/0
   199 ;; Data sizes:     COMRAM   BANK0   BANK1   BANK2   BANK3   BANK4   BANK5
   200 ;;      Params:         2       0       0       0       0       0       0
   201 ;;      Locals:         2       0       0       0       0       0       0
   202 ;;      Temps:          1       0       0       0       0       0       0
   203 ;;      Totals:         5       0       0       0       0       0       0
   204 ;;Total ram usage:        5 bytes
   205 ;; Hardware stack levels used: 1
   206 ;; Hardware stack levels required when called: 1
   207 ;; This function calls:
   208 ;;		Nothing
   209 ;; This function is called by:
   210 ;;		_main
   211 ;; This function uses a non-reentrant model
   212 ;;
   213                           
   214                           	psect	text1
   215  00004A                     __ptext1:
   216                           	callstack 0
   217  00004A                     _delay:
   218                           	callstack 29
   219  00004A                     
   220                           ;interrupt.c: 25:     for (int i=0;i<=ms;i++){
   221  00004A  0E00               	movlw	0
   222  00004C  6E05               	movwf	(delay@i+1)^0,c
   223  00004E  0E00               	movlw	0
   224  000050  6E04               	movwf	delay@i^0,c
   225  000052  EF2D  F000         	goto	l746
   226  000056                     l744:
   227                           
   228                           ;interrupt.c: 27:     }
   229  000056  4A04               	infsnz	delay@i^0,f,c
   230  000058  2A05               	incf	(delay@i+1)^0,f,c
   231  00005A                     l746:
   232  00005A  5004               	movf	delay@i^0,w,c
   233  00005C  5C01               	subwf	delay@ms^0,w,c
   234  00005E  5002               	movf	(delay@ms+1)^0,w,c
   235  000060  0A80               	xorlw	128
   236  000062  6E03               	movwf	??_delay^0,c
   237  000064  5005               	movf	(delay@i+1)^0,w,c
   238  000066  0A80               	xorlw	128
   239  000068  5803               	subwfb	??_delay^0,w,c
   240  00006A  B0D8               	btfsc	status,0,c
   241  00006C  EF3A  F000         	goto	u31
   242  000070  EF3C  F000         	goto	u30
   243  000074                     u31:
   244  000074  EF2B  F000         	goto	l744
   245  000078                     u30:
   246  000078  0012               	return		;funcret
   247  00007A                     __end_of_delay:
   248                           	callstack 0
   249                           
   250 ;; *************** function _ISR *****************
   251 ;; Defined at:
   252 ;;		line 17 in file "interrupt.c"
   253 ;; Parameters:    Size  Location     Type
   254 ;;		None
   255 ;; Auto vars:     Size  Location     Type
   256 ;;		None
   257 ;; Return value:  Size  Location     Type
   258 ;;                  1    wreg      void 
   259 ;; Registers used:
   260 ;;		status,2, status,0
   261 ;; Tracked objects:
   262 ;;		On entry : 0/0
   263 ;;		On exit  : 0/0
   264 ;;		Unchanged: 0/0
   265 ;; Data sizes:     COMRAM   BANK0   BANK1   BANK2   BANK3   BANK4   BANK5
   266 ;;      Params:         0       0       0       0       0       0       0
   267 ;;      Locals:         0       0       0       0       0       0       0
   268 ;;      Temps:          0       0       0       0       0       0       0
   269 ;;      Totals:         0       0       0       0       0       0       0
   270 ;;Total ram usage:        0 bytes
   271 ;; Hardware stack levels used: 1
   272 ;; This function calls:
   273 ;;		Nothing
   274 ;; This function is called by:
   275 ;;		Interrupt level 2
   276 ;; This function uses a non-reentrant model
   277 ;;
   278                           
   279                           	psect	intcode
   280  000008                     __pintcode:
   281                           	callstack 0
   282  000008                     _ISR:
   283                           	callstack 29
   284                           
   285                           ;incstack = 0
   286  000008  8206               	bsf	int$flags,1,c	;set compiler interrupt flag (level 2)
   287  00000A  ED3D  F000         	call	int_func,f	;refresh shadow registers
   288                           
   289                           	psect	intcode_body
   290  00007A                     __pintcode_body:
   291                           	callstack 29
   292  00007A                     int_func:
   293                           	callstack 29
   294  00007A  0006               	pop		; remove dummy address from shadow register refresh
   295  00007C                     
   296                           ;interrupt.c: 18:     if(INT0IF==1){
   297  00007C  A2F2               	btfss	4082,1,c	;volatile
   298  00007E  EF43  F000         	goto	i2u2_41
   299  000082  EF45  F000         	goto	i2u2_40
   300  000086                     i2u2_41:
   301  000086  EF46  F000         	goto	i2l740
   302  00008A                     i2u2_40:
   303  00008A                     
   304                           ;interrupt.c: 19:         PORTA=~PORTA;
   305  00008A  1E80               	comf	128,f,c	;volatile
   306  00008C                     i2l740:
   307                           
   308                           ;interrupt.c: 21:     INT0IF=0;
   309  00008C  92F2               	bcf	4082,1,c	;volatile
   310  00008E  9206               	bcf	int$flags,1,c	;clear compiler interrupt flag (level 2)
   311  000090  0011               	retfie		f
   312  000092                     __end_of_ISR:
   313                           	callstack 0
   314  0000                     
   315                           	psect	rparam
   316  0000                     
   317                           	psect	temp
   318  000006                     btemp:
   319                           	callstack 0
   320  000006                     	ds	1
   321  0000                     int$flags	set	btemp
   322  0000                     wtemp8	set	btemp+1
   323  0000                     ttemp5	set	btemp+1
   324  0000                     ttemp6	set	btemp+4
   325  0000                     ttemp7	set	btemp+8
   326                           
   327                           	psect	idloc
   328                           
   329                           ;Config register IDLOC0 @ 0x200000
   330                           ;	unspecified, using default values
   331  200000                     	org	2097152
   332  200000  FF                 	db	255
   333                           
   334                           ;Config register IDLOC1 @ 0x200001
   335                           ;	unspecified, using default values
   336  200001                     	org	2097153
   337  200001  FF                 	db	255
   338                           
   339                           ;Config register IDLOC2 @ 0x200002
   340                           ;	unspecified, using default values
   341  200002                     	org	2097154
   342  200002  FF                 	db	255
   343                           
   344                           ;Config register IDLOC3 @ 0x200003
   345                           ;	unspecified, using default values
   346  200003                     	org	2097155
   347  200003  FF                 	db	255
   348                           
   349                           ;Config register IDLOC4 @ 0x200004
   350                           ;	unspecified, using default values
   351  200004                     	org	2097156
   352  200004  FF                 	db	255
   353                           
   354                           ;Config register IDLOC5 @ 0x200005
   355                           ;	unspecified, using default values
   356  200005                     	org	2097157
   357  200005  FF                 	db	255
   358                           
   359                           ;Config register IDLOC6 @ 0x200006
   360                           ;	unspecified, using default values
   361  200006                     	org	2097158
   362  200006  FF                 	db	255
   363                           
   364                           ;Config register IDLOC7 @ 0x200007
   365                           ;	unspecified, using default values
   366  200007                     	org	2097159
   367  200007  FF                 	db	255
   368                           
   369                           	psect	config
   370                           
   371                           ; Padding undefined space
   372  300000                     	org	3145728
   373  300000  FF                 	db	255
   374                           
   375                           ;Config register CONFIG1H @ 0x300001
   376                           ;	unspecified, using default values
   377                           ;	Oscillator Selection bits
   378                           ;	OSC = 0x7, unprogrammed default
   379                           ;	Fail-Safe Clock Monitor Enable bit
   380                           ;	FCMEN = 0x0, unprogrammed default
   381                           ;	Internal/External Oscillator Switchover bit
   382                           ;	IESO = 0x0, unprogrammed default
   383  300001                     	org	3145729
   384  300001  07                 	db	7
   385                           
   386                           ;Config register CONFIG2L @ 0x300002
   387                           ;	unspecified, using default values
   388                           ;	Power-up Timer Enable bit
   389                           ;	PWRT = 0x1, unprogrammed default
   390                           ;	Brown-out Reset Enable bits
   391                           ;	BOREN = 0x3, unprogrammed default
   392                           ;	Brown-out Reset Voltage bits
   393                           ;	BORV = 0x3, unprogrammed default
   394  300002                     	org	3145730
   395  300002  1F                 	db	31
   396                           
   397                           ;Config register CONFIG2H @ 0x300003
   398                           ;	unspecified, using default values
   399                           ;	Watchdog Timer Enable bit
   400                           ;	WDT = 0x1, unprogrammed default
   401                           ;	Watchdog Timer Postscale Select bits
   402                           ;	WDTPS = 0xF, unprogrammed default
   403  300003                     	org	3145731
   404  300003  1F                 	db	31
   405                           
   406                           ; Padding undefined space
   407  300004                     	org	3145732
   408  300004  FF                 	db	255
   409                           
   410                           ;Config register CONFIG3H @ 0x300005
   411                           ;	unspecified, using default values
   412                           ;	PORTB A/D Enable bit
   413                           ;	PBADEN = 0x1, unprogrammed default
   414                           ;	Low-Power Timer 1 Oscillator Enable bit
   415                           ;	LPT1OSC = 0x0, unprogrammed default
   416                           ;	MCLR Pin Enable bit
   417                           ;	MCLRE = 0x1, unprogrammed default
   418  300005                     	org	3145733
   419  300005  82                 	db	130
   420                           
   421                           ;Config register CONFIG4L @ 0x300006
   422                           ;	unspecified, using default values
   423                           ;	Stack Full/Underflow Reset Enable bit
   424                           ;	STVREN = 0x1, unprogrammed default
   425                           ;	Single-Supply ICSP Enable bit
   426                           ;	LVP = 0x1, unprogrammed default
   427                           ;	Boot Block Size Select bit
   428                           ;	BBSIZ = 0x0, unprogrammed default
   429                           ;	Extended Instruction Set Enable bit
   430                           ;	XINST = 0x0, unprogrammed default
   431                           ;	Background Debugger Enable bit
   432                           ;	DEBUG = 0x1, unprogrammed default
   433  300006                     	org	3145734
   434  300006  85                 	db	133
   435                           
   436                           ; Padding undefined space
   437  300007                     	org	3145735
   438  300007  FF                 	db	255
   439                           
   440                           ;Config register CONFIG5L @ 0x300008
   441                           ;	unspecified, using default values
   442                           ;	Code Protection bit
   443                           ;	CP0 = 0x1, unprogrammed default
   444                           ;	Code Protection bit
   445                           ;	CP1 = 0x1, unprogrammed default
   446                           ;	Code Protection bit
   447                           ;	CP2 = 0x1, unprogrammed default
   448                           ;	Code Protection bit
   449                           ;	CP3 = 0x1, unprogrammed default
   450  300008                     	org	3145736
   451  300008  0F                 	db	15
   452                           
   453                           ;Config register CONFIG5H @ 0x300009
   454                           ;	unspecified, using default values
   455                           ;	Boot Block Code Protection bit
   456                           ;	CPB = 0x1, unprogrammed default
   457                           ;	Data EEPROM Code Protection bit
   458                           ;	CPD = 0x1, unprogrammed default
   459  300009                     	org	3145737
   460  300009  C0                 	db	192
   461                           
   462                           ;Config register CONFIG6L @ 0x30000A
   463                           ;	unspecified, using default values
   464                           ;	Write Protection bit
   465                           ;	WRT0 = 0x1, unprogrammed default
   466                           ;	Write Protection bit
   467                           ;	WRT1 = 0x1, unprogrammed default
   468                           ;	Write Protection bit
   469                           ;	WRT2 = 0x1, unprogrammed default
   470                           ;	Write Protection bit
   471                           ;	WRT3 = 0x1, unprogrammed default
   472  30000A                     	org	3145738
   473  30000A  0F                 	db	15
   474                           
   475                           ;Config register CONFIG6H @ 0x30000B
   476                           ;	unspecified, using default values
   477                           ;	Configuration Register Write Protection bit
   478                           ;	WRTC = 0x1, unprogrammed default
   479                           ;	Boot Block Write Protection bit
   480                           ;	WRTB = 0x1, unprogrammed default
   481                           ;	Data EEPROM Write Protection bit
   482                           ;	WRTD = 0x1, unprogrammed default
   483  30000B                     	org	3145739
   484  30000B  E0                 	db	224
   485                           
   486                           ;Config register CONFIG7L @ 0x30000C
   487                           ;	unspecified, using default values
   488                           ;	Table Read Protection bit
   489                           ;	EBTR0 = 0x1, unprogrammed default
   490                           ;	Table Read Protection bit
   491                           ;	EBTR1 = 0x1, unprogrammed default
   492                           ;	Table Read Protection bit
   493                           ;	EBTR2 = 0x1, unprogrammed default
   494                           ;	Table Read Protection bit
   495                           ;	EBTR3 = 0x1, unprogrammed default
   496  30000C                     	org	3145740
   497  30000C  0F                 	db	15
   498                           
   499                           ;Config register CONFIG7H @ 0x30000D
   500                           ;	unspecified, using default values
   501                           ;	Boot Block Table Read Protection bit
   502                           ;	EBTRB = 0x1, unprogrammed default
   503  30000D                     	org	3145741
   504  30000D  40                 	db	64
   505                           tosu	equ	0xFFF
   506                           tosh	equ	0xFFE
   507                           tosl	equ	0xFFD
   508                           stkptr	equ	0xFFC
   509                           pclatu	equ	0xFFB
   510                           pclath	equ	0xFFA
   511                           pcl	equ	0xFF9
   512                           tblptru	equ	0xFF8
   513                           tblptrh	equ	0xFF7
   514                           tblptrl	equ	0xFF6
   515                           tablat	equ	0xFF5
   516                           prodh	equ	0xFF4
   517                           prodl	equ	0xFF3
   518                           indf0	equ	0xFEF
   519                           postinc0	equ	0xFEE
   520                           postdec0	equ	0xFED
   521                           preinc0	equ	0xFEC
   522                           plusw0	equ	0xFEB
   523                           fsr0h	equ	0xFEA
   524                           fsr0l	equ	0xFE9
   525                           wreg	equ	0xFE8
   526                           indf1	equ	0xFE7
   527                           postinc1	equ	0xFE6
   528                           postdec1	equ	0xFE5
   529                           preinc1	equ	0xFE4
   530                           plusw1	equ	0xFE3
   531                           fsr1h	equ	0xFE2
   532                           fsr1l	equ	0xFE1
   533                           bsr	equ	0xFE0
   534                           indf2	equ	0xFDF
   535                           postinc2	equ	0xFDE
   536                           postdec2	equ	0xFDD
   537                           preinc2	equ	0xFDC
   538                           plusw2	equ	0xFDB
   539                           fsr2h	equ	0xFDA
   540                           fsr2l	equ	0xFD9
   541                           status	equ	0xFD8

Data Sizes:
    Strings     0
    Constant    0
    Data        0
    BSS         0
    Persistent  0
    Stack       0

Auto Spaces:
    Space          Size  Autos    Used
    COMRAM           94      5       5
    BANK0           160      0       0
    BANK1           256      0       0
    BANK2           256      0       0
    BANK3           256      0       0
    BANK4           256      0       0
    BANK5           256      0       0

Pointer List with Targets:

    None.

Critical Paths under _main in COMRAM

    _main->_delay

Critical Paths under _ISR in COMRAM

    None.

Critical Paths under _main in BANK0

    None.

Critical Paths under _ISR in BANK0

    None.

Critical Paths under _main in BANK1

    None.

Critical Paths under _ISR in BANK1

    None.

Critical Paths under _main in BANK2

    None.

Critical Paths under _ISR in BANK2

    None.

Critical Paths under _main in BANK3

    None.

Critical Paths under _ISR in BANK3

    None.

Critical Paths under _main in BANK4

    None.

Critical Paths under _ISR in BANK4

    None.

Critical Paths under _main in BANK5

    None.

Critical Paths under _ISR in BANK5

    None.

Call Graph Tables:

 ---------------------------------------------------------------------------------
 (Depth) Function   	        Calls       Base Space   Used Autos Params    Refs
 ---------------------------------------------------------------------------------
 (0) _main                                                 0     0      0     198
                              _delay
 ---------------------------------------------------------------------------------
 (1) _delay                                                5     3      2     198
                                              0 COMRAM     5     3      2
 ---------------------------------------------------------------------------------
 Estimated maximum stack depth 1
 ---------------------------------------------------------------------------------
 (Depth) Function   	        Calls       Base Space   Used Autos Params    Refs
 ---------------------------------------------------------------------------------
 (2) _ISR                                                  0     0      0       0
 ---------------------------------------------------------------------------------
 Estimated maximum stack depth 2
 ---------------------------------------------------------------------------------

 Call Graph Graphs:

 _main (ROOT)
   _delay

 _ISR (ROOT)

 Address spaces:
Name               Size   Autos  Total    Cost      Usage
BITCOMRAM           5E      0       0       0        0.0%
EEDATA             100      0       0       0        0.0%
NULL                 0      0       0       0        0.0%
CODE                 0      0       0       0        0.0%
COMRAM              5E      5       5       1        5.3%
STACK                0      0       0       2        0.0%
ABS                  0      0       0       3        0.0%
BITBANK0            A0      0       0       4        0.0%
BANK0               A0      0       0       5        0.0%
BITBANK1           100      0       0       6        0.0%
BANK1              100      0       0       7        0.0%
BITBANK2           100      0       0       8        0.0%
BANK2              100      0       0       9        0.0%
BITBANK3           100      0       0      10        0.0%
BANK3              100      0       0      11        0.0%
BITBANK4           100      0       0      12        0.0%
BANK4              100      0       0      13        0.0%
BITBANK5           100      0       0      14        0.0%
BANK5              100      0       0      15        0.0%
BIGRAM             5FF      0       0      16        0.0%
DATA                 0      0       0      17        0.0%
BITSFR_3             0      0       0     200        0.0%
SFR_3                0      0       0     200        0.0%
BITSFR_2             0      0       0     200        0.0%
SFR_2                0      0       0     200        0.0%
BITSFR_1             0      0       0     200        0.0%
SFR_1                0      0       0     200        0.0%
BITSFR               0      0       0     200        0.0%
SFR                  0      0       0     200        0.0%


Microchip Technology PIC18 Macro Assembler V2.32 build 20210201212658 
Symbol Table                                                                                   Mon Jan 17 12:07:46 2022

                     l40 0078                       l25 0024                       u30 0078  
                     u31 0074                      l742 004A                      l750 001E  
                    l744 0056                      l760 0036                      l752 0020  
                    l746 005A                      l754 0022                      l756 0028  
                    l748 0012                      l758 0034                      _ISR 0008  
                   ?_ISR 0001                     _GIEH 007F97                     _PEIE 007F96  
                   i2l34 008E                     _main 0012                     btemp 0006  
                   start 000E             ___param_bank 000000                    ??_ISR 0001  
                  ?_main 0001                    i2l740 008C                    i2l736 007C  
                  i2l738 008A                    _PORTA 000F80                    _PORTC 000F82  
                  _TRISA 000F92                    _TRISC 000F94                    _delay 004A  
                  ttemp5 0007                    ttemp6 000A                    ttemp7 000E  
                  status 000FD8                    wtemp8 0007          __initialization 0092  
           __end_of_main 004A                   ??_main 0006            __activetblptr 000000  
                 ?_delay 0001                   _ADCON1 000FC1                   _INT0IE 007F94  
                 _INT0IF 007F91                   i2u2_40 008A                   i2u2_41 0086  
                 delay@i 0004                   isa$std 000001               __accesstop 0060  
__end_of__initialization 0092            ___rparam_used 000001           __pcstackCOMRAM 0001  
          __end_of_delay 007A                  ??_delay 0003                  __Hparam 0000  
                __Lparam 0000                  __pcinit 0092                  __ramtop 0600  
                __ptext0 0012                  __ptext1 004A             __size_of_ISR 008A  
                delay@ms 0001           __pintcode_body 007A     end_of_initialization 0092  
                int_func 007A      start_initialization 0092              __end_of_ISR 0092  
              __pintcode 0008           __size_of_delay 0030                 __Hrparam 0000  
               __Lrparam 0000            __size_of_main 0038                 isa$xinst 000000  
               int$flags 0006                 intlevel2 0000  
